:100000000EC01BC01AC019C02BC017C016C015C027
:1000100014C013C012C011C010C00FC00EC01124F4
:100020001FBECFEDCDBF20E0A0E6B0E001C01D9225
:10003000A736B207E1F733D16EC2E2CFE199FECF26
:1000400090E09FBB8EBBE09A8DB30895E199FECFFF
:100050001CBA90E09FBB8EBB6DBBE29AE19A0895FB
:100060001F920F920FB60F9211242F933F938F93ED
:100070009F93AF93BF9380E28FBD8091620091E028
:10008000980F909362008F7009F047C080916000D4
:10009000909161009C012F5F3F4F3093610020934E
:1000A0006000803F910578F4809163009091640036
:1000B000A0916500B091660080FF2FC098B382E0E8
:1000C000892788BB2AC0109261001092600080913D
:1000D000630090916400A0916500B0916600B695B0
:1000E000A795979587958093630090936400A0935C
:1000F0006500B09366008091630090916400A091C8
:100100006500B0916600892B8A2B8B2B31F489B75F
:100110008B7F89BF80B5886080BDBF91AF919F9173
:100120008F913F912F910F900FBE0F901F901895B8
:100130006093630070936400809365009093660001
:100140008091630090916400A0916500B091660079
:10015000892B8A2B8B2B51F080B5877F80BD81E066
:1001600080BF8FEF8FBD89B7846089BF089525E078
:100170003FE042EF4A95F1F73A95E1F72A95D1F73A
:100180000895A39A80B58E7F80BD80E887B987E8FF
:1001900086B9089580B58E7F80BD87B1836887B9A1
:1001A000369A3699FECF80B5816080BD84B195B115
:1001B0000895AF92BF92CF92DF92EF92FF920F938A
:1001C0001F93CF93DF93EC01062F10E0780121E01D
:1001D000E21AF1081E141F0454F135C090E0292FD3
:1001E00030E0220F331F6E01C20ED31EF601A08134
:1001F000B1812E5F3F4F5E01A20EB31EF50120813B
:1002000031812A173B0730F4F60131832083F50151
:10021000B183A0839F5F292F30E026173707FCF2B8
:100220008F5F282F30E02E153F0524F00CC020E012
:1002300030E080E0B801621B730B61507109161643
:10024000170664F2EDCF642F70E0061B170B6017E2
:10025000710794F480E090E0FE01E40FF11DE40FDB
:10026000F11D20813181820F931F4F5F242F30E0D9
:10027000201731078CF302C080E090E09801261B24
:10028000370BB90134D1CB01DF91CF911F910F9181
:10029000FF90EF90DF90CF90BF90AF900895CF93F5
:1002A000DF93CDB7DD27C952CDBFF894B99ABA987C
:1002B000BC98C29AC49AB89A89B78B7F89BF789440
:1002C00065E170E080E090E033DF83E88ABD81E0A3
:1002D00083BF80BFB3DE082F853608F001E051DF11
:1002E000512C10E0612C712CD12CA12CB12C812C23
:1002F000912CEE24E394F12CC12C19A60F2EF4E1DD
:100300002F2E312CF02D57C0C401B101F0D07C014B
:1003100041DFF701EE0FFF1F21E030E02C0F3D1F02
:10032000E20FF31F91838083EF28E1F535E1831617
:100330009104C0F145E064E1CE0101963ADF8F32CD
:1003400021E0920728F439A5311102C021E029A744
:100350008E32914028F489A5813009F0ADC009C0E2
:1003600029A5213041F465E070E080E090E0E0DE16
:100370000DC033E039A789A5823041F465E170E012
:1003800080E090E0D5DE0EC023E029A739A5333008
:1003900049F465E570E080E090E0CADE6894CC2422
:1003A000C1F800E08FEF881A980A2FEFA21AB20A5C
:1003B00080E090E07C013DE2A31631E0B30660F0FE
:1003C000C11085C061E070E080E090E0B1DE512EA8
:1003D000CC24C39400E07BC0DD2011F0DA945CC033
:1003E00046B2842D80958471482EC11030C087118B
:1003F00077C0639482E0861508F06EC020E1421257
:100400000EC0043610F40F5F67C061E070E080E05A
:1004100090E08EDE0F2EFAE0DF2EF02D5DC034E08E
:10042000431205C0002309F455C0015053C084E1B4
:10043000481252C0612F81E009DE65E070E080E083
:1004400090E076DE0F2EFAE0DF2EF02D4EC0442035
:1004500001F122E0C2120CC065E570E080E090E09E
:1004600067DE0F2EFAE0DF2EF02D16C0742C612C03
:1004700031E0C31210C061E070E080E090E058DE2F
:10048000052DA12CB12CC12C0F2EFAE0DF2EF02D62
:1004900003C0D12C01C0D12C101708F41F5F011725
:1004A00008F4115019BD63DEC701019624E1E2167C
:1004B000F10409F07FCF28CF39A5323009F066CF9B
:1004C00063CF46B2842D80958471482EC0CFD11061
:1004D00085CFF7CF742CCCCF411007C0742CDCCF64
:1004E0008111C4CF782E612CD7CF742CD5CFAA1B05
:1004F000BB1B51E107C0AA1FBB1FA617B70710F00F
:10050000A61BB70B881F991F5A95A9F78095909540
:0A051000BC01CD010895F894FFCF5F
:00000001FF
